:020000040800F2
:1000000018070020D10000089D15000831130008D2
:1000100000000000000000000000000000000000E0
:10002000000000000000000000000000B11F0008F8
:1000300000000000000000000F1700086D210008FC
:100040000101000801010008010100080101000888
:1000500001010008AD0D00080101000801010008C0
:100060000101000801010008070C00080101000857
:100070000101000801010008010100080101000858
:100080000101000801220008010100080101000827
:100090000101000801010008010100080101000838
:1000A000010100080101000801010008A92300085E
:1000B000E52300080D2400080101000803488546D7
:1000C00000F046FC00480047A13500081807002052
:1000D0000C4880F308880C480168090E0B4A9142CD
:1000E00005D10B480B4901600B480C4901600C48D5
:1000F00080470C480047FEE7FEE7FEE7FEE7FEE725
:10010000FEE7000018070020040000001F000000A8
:100110001810024001000000000001400000000033
:1001200085210008BD00000830B50B4601460020BF
:100130002022012409E00D46D5409D4205D31D46ED
:100140009540491B2546954040191546521E002DE5
:10015000F1DC30BD70B500242546002801DA012409
:100160004042002901DA01254942FFF7DDFFAC4298
:1001700000D04042002C00D0494270BD30B5054649
:100180000020034600E05B1C934205D2EC5CC85C97
:10019000201A01D1002CF6D130BDF8B502464A40F4
:1001A000D40F42004B0052085B089A4202D202462A
:1001B000084611464A0023D0C30D4A00DDB2120E94
:1001C000AD1A202D35DA49020126490AF6058A19A9
:1001D000002C00D0524220214F1B1146B9402A4129
:1001E0001018C20D9A4221D0002C17D0012D08DC26
:1001F000DA05801AD20F8019D207DBB200F0C2F9FB
:10020000F8BDDA05801A012340001B06C0188018CB
:100210005A428018CA0F1043490007E04908C20734
:100220001143DA05801A80194008801800F0A2F9FD
:10023000F8BD61000122511A001BF7E70122D20725
:100240005140AAE70122D2075040A6E7024670B506
:100250004A40D30FDB0740002DD04A002AD0010EC0
:10026000140E000212020919400A520A8418E5010C
:1002700004465443000A120A2E045043A41942199A
:10028000200CC543AA18120C0125AD03521C5219AB
:1002900012047F39240400D0521C104301D44000C2
:1002A000491EC2B20C06C0092018401C4008802A12
:1002B00002D003E0002070BD40084000002900DAB1
:1002C0000020184370BD70B502464A40D50F40006B
:1002D0004A00ED0740085208002814D0002A12D026
:1002E000C40DD30D41020120C0055202490A520A31
:1002F000E41A091812187D34914201D3641C00E0FD
:100300004900002C01DA002070BD0023914201D386
:10031000891A0343400849000028F7D100290AD070
:10032000914202D10121C90705E0914201D2012188
:1003300001E00121C943E005C018401900F01AF995
:1003400070BD0000F0B50C465C4085B0E40FE407DA
:1003500003944C000026640859009446490802465C
:100360000296224321D062460A431ED06200570DF6
:100370004A000E032303550D012402462C4924058F
:10038000781B1B0B360B4018234326436146009015
:100390001C46501AB44103D30098401C009002E060
:1003A000921800985B41002803DA0020014605B04E
:1003B000F0BD0020012109050746864611E064468C
:1003C0001D46141BB54106D36546521BB341744606
:1003D00007430C43A646CD07400849082843921816
:1003E0005B4105460D43EAD11046184313D06046E1
:1003F000194650407140084306D06046101AB34178
:1004000006D20122002306E000220123DB0702E0DE
:100410000122D2435310009874460105381C6141F3
:10042000029C039D0019694100F0E5F8BFE7000058
:10043000FD03000010B500229623114600F0A2F83B
:1004400010BD00000EB5C217C10F5040CA074018BA
:100450000021054B0293019200910A460B4600F0E1
:10046000D7F803B000BD000033040000C20F410004
:1004700040020123400ADB05D207090EC0187F297C
:1004800001DA00207047962903DC9623591AC840E8
:1004900001E096398840002AF4D040427047C20FEC
:1004A000D207400040080BD0C10D0723DB01C9185B
:1004B00040020905400A1143C20840071143704732
:1004C000002001467047CB0FDB07490010B54908F3
:1004D00002460A4307D00A0D07240903E401090B69
:1004E000121B002A01DC002010BDC900440F0C4380
:1004F000C100E018D205801800F03CF810BD0000E3
:100500000122D207002800DB101A002900DB511A53
:1005100088427047F0B51FB40646002082B00546F9
:100520004024019100901BE0019922460F4630467D
:1005300000F030FA049A059B801A994110D31046B6
:100540001946224600F016FA361A8F4101972246C4
:1005500001200021009F00F00DFA38184D41009055
:100560002046641E0028DFDC019B009829463246A5
:1005700007B0F0BD002904DA401C490001D1400851
:100580004000704770B40024050C05D1102400040D
:1005900002D1002921D01124050E01D10002083416
:1005A000050F01D10001241D850F01D18000A41C7D
:1005B000002801DB4000641C002908D020252E1BE8
:1005C0000D46F540A14000D0012129430843010612
:1005D0001B1B000ADB1D02D5002070BC7047DB0529
:1005E000181880180029F8DA401C4900F5D170BCB1
:1005F00040084000704710B5002B08DA0024401C6A
:10060000614192185B411A4301D14008400010BD7E
:10061000F0B51FB482B005460C0003D0084602F0C6
:1006200031FB02E002F02EFB203002460090214612
:10063000284600F09FF9049B059A04460F4618438C
:100640001143084314D0184610431BD00098402192
:100650000A1A1846059900F09DF905460E46009ABB
:100660000599049800F086F9084305D0012004E0BC
:100670002046394607B0F0BD0020C11705430E43A0
:100680002C43374300990E986305401A7905E40A14
:1006900000220C43FD0A0A3002D500200146E9E79A
:1006A0000105101969410C9C0D9D00196941FFF766
:1006B000A2FFDFE7F0B507460846584087B0C00FF5
:1006C000049048000E46590040084908BC1A884169
:1006D00005D2384631461E4617460B46024658009C
:1006E000400810434CD0300D039040055900400D98
:1006F000490D0590401A0290402872DA1803012132
:10070000000B09050843019004980092002805D0C9
:1007100001995242002088410092019002984021A4
:100720000A1A0199009800F025F905460C466B4617
:1007300007CB00F040F9C0197141039A0E0D002358
:10074000D71756401A467A40164344D0049A002AD6
:100750002DD0029A012A039A15DC1205C01A914184
:1007600001263605001C7141D20F059ED207009369
:10077000019202962A462346FFF74AFF07B0F0BDD2
:1007800038463146FAE71605224A0F46B218C01A13
:10079000B74101210905001C4F4100187F41114656
:1007A00018187941E20F10436D19644113E0E20714
:1007B0006D0815436408C2071443039A0126120505
:1007C000C01A91413605001C7141CE0740083043E4
:1007D0004908C01851412A462346FFF70CFFCDE7D0
:1007E000FFE7049801224000C117121A00238B4131
:1007F00004983146C417381AA141EEE730B40124F9
:10080000E407634030BC55E730B40124E40761409D
:1008100030BC4FE70000E0FFF0B51FB488B00B9983
:100820000998002448400999C00F490049080991D6
:10083000C0070B990090490049080B910999089845
:10084000A64608431CD00B990A98084318D009986B
:1008500001244000420D4800410D09982405000381
:10086000000B204309900B980003000B20430B90D2
:1008700050181C494018002201901446104605E00B
:10088000002001460DB0F0BD032801DA034600E068
:1008900003239C46C11A0AAE0AE05F0008ADED5B77
:1008A0004F00F75B7D430027AA187C41491C5B1E63
:1008B0006145F2DD410004AB5A522104120C0A4397
:1008C000240C401C0828DFDB019802900099704638
:1008D00001910090059B049A07990698FFF798FEEE
:1008E000D0E700000DFCFFFF4A0009030123090BBC
:1008F0001B0519430A4B10B5520D9A4202DA00202B
:10090000014610BD064B34339A4203DC9A1A00F0BC
:1009100041F810BD034BD21800F02CF810BD0000B8
:10092000FF030000CDFBFFFF10B5002904DB01240D
:10093000E40740428C412146002B04DB1C46012386
:10094000DB075242A341994200D1904210BD000002
:10095000064C0125064E05E0E36807CC2B430C3C12
:1009600098471034B442F7D3FFF7ACFB5437000874
:100970007437000810B5202A04DB0146203A914064
:10098000002010BD914020239C1A0346E3401943E8
:10099000904010BD10B5202A04DB0846203AD04014
:1009A000002110BD0B46D340D0402024A21A914014
:1009B0000843194610BD10B5202A06DBCB170846A0
:1009C000203A1041C1170B4306E00B461341D040BB
:1009D0002024A21A91400843194610BDFFB587B0E4
:1009E00004460E46109D00212068FFF789FD03D8BC
:1009F00001212420015502E0002124200155206816
:100A0000FFF734FDC1B2252001557B492068FFF76F
:100A10001DFC0290FFF72AFD64210390FFF79AFB6B
:100A20002620015500200690012005E0325C069941
:100A30005118C9B20691401C0828F7DB0698C0433C
:100A4000401CC0B20690317A0698884210D1B17825
:100A50000902F2788818FFF7F5FC0022674B019134
:100A60000090FFF76FFC03910290FFF72CFDA06050
:100A70000027012004E00A99095CC919CFB2401C83
:100A80000828F8DBF843401CC7B20A98007A87426E
:100A900012D10A9989790A020A99C9795018FFF77F
:100AA000D1FC0022564B01910090FFF74BFC0391C3
:100AB0000290FFF708FD20610020059000BF05E0CF
:100AC0002A5C0599511889B20591401C1D28F7DB55
:100AD00005980012A97F88421CD10598C0B2E97F11
:100AE000884217D1287B0002697B4018E061A87B0F
:100AF0000002E97B401820627D210901E0698842FB
:100B000001DD0846E0617D210901206A884201DD9E
:100B10000846206200200490012006E009990A5C42
:100B200004995118C9B20491401C0828F6DB0498B6
:100B3000C043401CC0B204900999097A04988842C5
:100B400012D1099989780A020999C9785018FFF7D2
:100B500079FC0022294B01910090FFF7F3FB0391F0
:100B60000290FFF7B0FCE0606068FFF77FFCC1B265
:100B70002720015520496068FFF768FB0290FFF7C6
:100B800075FC64210390FFF7E5FA28200155A06861
:100B9000FFF76CFCC1B2292001551749A068FFF787
:100BA00055FB0290FFF762FC64210390FFF7D2FA35
:100BB0002A200155FF212B2001552C2001552D20E5
:100BC00001552E2001552F20015530200155FF20C1
:100BD000A061A08B0004010E33200155217F342039
:100BE0000155208C0004010E35200155208CC1B226
:100BF000362001550BB0F0BD0000C842000059403E
:100C000000408F40704710B50120400200F024F8EA
:100C10000120400200F002F810BD00000121090788
:100C20000140002902D00349486001E002494860C0
:100C3000704700000004024000000240002904D078
:100C4000026801231A43026003E00268014B1A4064
:100C500002607047FEFF00000146002000220123D1
:100C60001B070B40002B02D0064B1A6801E0064B15
:100C70001A6813460B40002B01D0012000E0002031
:100C800070470000000402400000024010B500223E
:100C900002680D4B1A400C6A8B6823430C6923438E
:100CA0004C6923438C692343CC6923434C6A234317
:100CB0008C6A23431A430260CB6843600B688360ED
:100CC0004B68C36010BD00000F80FFFF10B50B4ADA
:100CD000904200D100E000BFA82212580B0F9C00E8
:100CE0000F23A3409A43A8231A50A82212580B019D
:100CF0001B091A43A8231A5010BD0000000002402F
:100D00001CB5084800F04CFA07480849084B094A46
:100D10000091019008490348FFF760FE014801F087
:100D200048F91CBD5C000020D40100201401002003
:100D3000D4000020940100209400002003490860A2
:100D400000BF024909680029FBD170473C00002020
:100D50000EE00021084A116005E000BF064909685D
:100D6000491C054A1160044909680429F5D3401E4D
:100D70000028EED170470000400000200FE0002165
:100D8000084A116005E000BF06490968491C054A88
:100D9000116004490968044A9142F4D3401E0028B6
:100DA000EDD17047440000200B11000010B5012068
:100DB00000F026F8002808D001200649087000F04D
:100DC00019F805A001F04EFF02E003200849486130
:100DD00010BD000054000020425554544F4E305F67
:100DE00049525148616E646C65720D0A0000000042
:100DF00000040140014948617047000000040140BF
:100E000001460020044A52690A40002A01D001200C
:100E100000E000207047000000040140002806D0D8
:100E20000649096810221143044A116005E003498C
:100E3000096810229143014A116070470020024066
:100E400001460020044A10684008400002460A4358
:100E50001046014A10607047002002401CB5012274
:100E600003210920C00600F06BF9012202210920AC
:100E7000C00600F065F90C2000900221684601715F
:100E80000321417100218171C17169460920C006A9
:100E900000F00EF900220721824800F051F90022EB
:100EA0000621804800F04CF9C020009002216846DD
:100EB00001710321417100218171C1716946794835
:100EC00000F0F6F801220521774800F039F90122F7
:100ED0000421754800F034F9302000900221684662
:100EE00001710321417100218171C17169466E4810
:100EF00000F0DEF8042201210920C00600F020F9EC
:100F0000042200210920C00600F01AF903200090F5
:100F10000221684601710321417100218171C17173
:100F200069460920C00600F0C3F8022211465F4856
:100F300000F006F902220C215B4800F001F90420C0
:100F400000900221684601710321417100218171E5
:100F5000C1716946554800F0ABF8012000030090CC
:100F60000221684601710321417100218171C17123
:100F700069464D4800F09CF8052211460920C0063C
:100F800000F0DEF8052204210920C00600F0D8F8A0
:100F90003020009002216846017103214171002137
:100FA0008171C17169460920C00600F081F80122F3
:100FB00007213D4800F0C4F8012206213A4800F01C
:100FC000BFF8C020009002216846017103214171E1
:100FD00000218171C1716946334800F069F801222E
:100FE0000921314800F0ACF8012208212E4800F018
:100FF000A7F8032000020090022168460171032136
:10100000417100218171C1716946274800F050F893
:101010000320800200900021684601714171C17176
:101020006946204800F044F8FF200130009001217B
:1010300068460171002141710121C1710021817156
:1010400069460920C00600F033F80C200090012109
:1010500068460171002141710121C1710021817136
:101060006946114800F024F804210F4800F096F872
:1010700008210D4800F092F80120C00300900121E2
:1010800068460171002141710121C1710021817106
:101090006946044800F00CF80121C903014800F03A
:1010A0007DF81CBD0004004800080048000C004802
:1010B000F0B50A4600210023002400BF3DE00125D1
:1010C0008D402B4615681D402C469C4234D1157925
:1010D000012D02D01579022D16D185684F00032607
:1010E000BE40B543856055794E00B54086683543AE
:1010F0008560858801268E40B543858085889679F0
:101100008E40B6B23543858005684F000326BE4049
:10111000B543056015794E00B54006683543056056
:10112000C5684F000326BE40B543C560D5794E0063
:10113000B540C6683543C560491C1029BFD3F0BD12
:10114000F0B5002300244D07EE0E1546B5402B46A2
:10115000CD10AE0005462035AD594E07F70E0F26CF
:10116000BE40B543CE10B60007462037BD51CD1066
:10117000AE003D46AD591D432C46CD10AD003E4658
:101180007451F0BD02460020138A0B40002B01D0A1
:10119000012000E0002070470185704781617047A1
:1011A0007FB50446C820FFF7C9FD012189024E48DA
:1011B000FFF7E8FF312108550121C9024A48FFF72E
:1011C000E1FF322108553120005D002801D10120C6
:1011D00000E000203221095D002901D1012100E059
:1011E00000210840002801D00020A0613120005DCE
:1011F000002801D1012000E000203221095D0129F1
:1012000000D100E000210840002801D00120A061A9
:101210003120005D012800D100E000203221095D6D
:10122000002901D1012100E000210840002801D05F
:101230000220A0613120005D012800D100E00020E3
:101240003221095D012900D100E000210840002879
:1012500001D00320A061C820FFF770FD07222349B9
:10126000234801F0E9FCC820FFF768FD0922214965
:10127000214801F0E1FCC820FFF760FD09221F4969
:101280001F4801F0D9FCC820FFF758FD09221D496D
:101290001D4801F0D1FCC820FFF750FD0922194973
:1012A0001A4801F0C9FC3220FFF768FD3220012303
:1012B0000022211D0090204600F00BFD3220FFF798
:1012C0005DFD6068FFF7EBF805460E462068FFF706
:1012D000E6F802460B4601960095039102900CA099
:1012E00001F0C0FC7FBD000000040048D4360008B7
:1012F000004C0040F7360008001401403637000863
:10130000004800401B3700080050004000380140F2
:1013100074656D70657261747572653A25662C68C6
:10132000756D69646974793A25660D0A00000000DC
:1013300000BFFEE7F8B504460E46174600200090B1
:101340002070012080020921C9068861802522E0E1
:10135000012040020921C90688610120FFF7F8FC3D
:10136000384600F082F800900320FFF7F1FC0920D6
:10137000C006008A012189020840002802D0207896
:1013800028432070012040060921C90688610120F8
:10139000FFF7DEFC6D10002DDADC002E05D10120F8
:1013A00080060921C906886104E001208002092124
:1013B000C90688610120FFF7CBFC0120400209210A
:1013C000C90688610520FFF7C3FC012040060921FA
:1013D000C9068861C01388611420FFF7B9FC009822
:1013E000F8BD10B5012080020921C90688610120DD
:1013F000FFF7AEFC012040020921C90688610120E7
:10140000FFF7A6FC012080060921C90688610A2091
:10141000FFF79EFC012040060921C90688610A20C9
:10142000FFF796FC10BD10B5012040060921C90642
:1014300088610120FFF78CFC012080060921C90684
:1014400088610120FFF784FC012040020921C906C0
:1014500088610A20FFF77CFC012080020921C9066F
:1014600088610A20FFF774FC10BD70B504460025A2
:1014700009E02046611ECCB2002801D1042070BDD5
:101480000120FFF77BFC0920C006008A01214902E8
:1014900008400028EDD02846F1E770B50546002643
:1014A000802422E020462840002805D10120800623
:1014B0000921C906886104E0012080020921C906CA
:1014C00088610120FFF744FC012040020921C90680
:1014D00088610520FFF73CFC012040060921C90670
:1014E00088610120FFF734FC6410002CDADC012055
:1014F00080020921C9068861401088610120FFF738
:1015000027FC0920C006008A012189020840002822
:1015100000D00126012040060921C9068861142057
:10152000FFF716FC304670BD70B505460C460748FF
:1015300000F02EF8284600F01FF8204600F022F8B0
:1015400000F012F800F004F870BD000055550000DE
:101550000148024908607047CCCC000000300040D0
:1015600010B500F001F810BD01480249086070474D
:10157000AAAA0000003000400149486070470000FE
:101580000030004001498860704700000030004092
:10159000014908607047000000300040704708B5FE
:1015A0001C216846017001214170817000F03AF8F9
:1015B0001B216846017001214170817000F032F8F2
:1015C0001D216846017001214170817000F02AF8E8
:1015D0001D216846017001214170817000F022F8E0
:1015E0001D216846017001214170817000F01AF8D8
:1015F0001D216846017001214170817000F012F8D0
:101600001D216846017001214170817000F00AF8C7
:101610001D216846017001214170817000F002F8BF
:1016200008BD000000218278002A27D0184A032331
:101630001B02D21803789B109B00D15802789207A6
:10164000D30EFF229A400B469343194642789207E5
:10165000120E03789B07DB0E9A4011430C4A0323BA
:101660001B02D21803789B109B00D1500278D3063E
:10167000DB0E01229A40064B1A6007E00278D3067F
:10168000DB0E01229A40024B80331A607047000043
:1016900000E100E010B5002819DA1A4A03071B0F11
:1016A000083B9B089B00D2588307DC0EFF23A34016
:1016B0009A438B071B0E8407E40EA3401A43114B79
:1016C0000407240F083CA408A4001A5118E00E4A8D
:1016D00003231B02D21883089B00D2588307DC0E19
:1016E000FF23A3409A438B071B0E8407E40EA340FD
:1016F0001A43054B032424021B198408A4001A5121
:1017000010BD00001CED00E000E100E070477047F4
:10171000002905D0054A52690243044B5A6104E08E
:10172000024A52698243014B5A61704700100240DD
:10173000002905D0054AD2690243044BDA6104E06E
:10174000024AD2698243014BDA61704700100240BD
:10175000002905D0054A92690243044B9A6104E0CE
:10176000024A92698243014B9A617047001002401D
:101770001948006801210843174908600846406875
:101780001649084014494860084600681449084052
:1017900011490860084600680121890488430E4900
:1017A0000860084640683F21090488430A494860A8
:1017B0000846C06A00090001C8620846006B094972
:1017C0000840054908630846406B400840004863EC
:1017D0000020886070470000001002400CB8FF082D
:1017E000FFFFF6FEACFEF0FFFEB504460025002626
:1017F00000200290019000900027864840680C214C
:1018000008400546002D06D0042D07D0082D08D02D
:101810000C2D2CD128E0804820602BE07F482060F0
:1018200028E07C4840680F21890408400646794832
:1018300040680321C90308400290B00C861C02983E
:10184000002803D17648374647430BE07148C06A09
:101850000007000F401C019070480199FEF764FCDE
:1018600070430746276005E06E48206002E06A4842
:10187000206000BF00BF67484068F021084005466F
:101880002D096948405D009020680099C84060605B
:101890006048406807210902084005462D0A624851
:1018A000405D009061680098C140A1605948006B9C
:1018B000FF2101310840884202D05C48E0600DE021
:1018C00054484068012189030840884203D0A06839
:1018D0004008E06002E0A0688008E0604D48006BCE
:1018E00040210840402802D05148206102E00120F8
:1018F000C00320614748006B10210840102802D027
:101900004548606101E0206860614248006B8007E3
:10191000800F002802D1A068A06119E03D48006B4B
:101920008007800F012802D12068A06110E03948AB
:10193000006B8007800F022802D18003A06107E0BE
:101940003448006B8007800F032801D13248A06122
:101950003048006B032109040840002802D1A06828
:10196000E06120E02B48006B0321090408400121BD
:101970000904884202D12068E06114E02548006B28
:1019800003210904084001214904884202D1801042
:10199000E06108E01F48006B032109040840884209
:1019A00001D11D48E0611B48006B032189040840F8
:1019B000002802D1A068206220E01648006B0321B5
:1019C0008904084001218904884202D120682062EC
:1019D00014E01048006B0321890408400121C90468
:1019E000884202D10011206208E00A48006B0321FE
:1019F00089040840884201D1074820620548006BED
:101A000080210840802802D00648606200E06762BA
:101A1000FEBD00000010024000127A000024F40015
:101A200000093D00006CDC0214000020809FD500FE
:101A30001280000010B50246002100230020511141
:101A4000002902D10C4C23680BE0012902D10A4C79
:101A5000236A06E0022902D1074C636A01E0064CC2
:101A6000636BD106C90E01248C401C40002C01D0B0
:101A7000012000E0002010BD001002400248406834
:101A80000C21084070470000001002400146002071
:101A9000054A5068F02302469A43104602460A431C
:101AA0001046014A50607047001002400021024A6F
:101AB0009170114688707047001002400549096B0B
:101AC00010229143034A11631146096B01431163CC
:101AD000704700000010024001460020064A50688E
:101AE00007231B0202469A43104602460A43104649
:101AF000014A50607047000000100240002807D0E3
:101B000007490968012212061143054A116006E0DF
:101B100003490968012212069143014A1160704786
:101B200000100240074A52687B23DB039A43054BAF
:101B30005A601A46526803460B431A43014B5A60D7
:101B4000704700000010024001460020044AD06A9D
:101B50000009000102460A431046014AD06270475C
:101B60000010024001460020044A506880088000AE
:101B700002460A431046014A506070470010024076
:101B80000021010F012906D10E4A126B9208920022
:101B90000C4B1A6310E0022907D10A4A126B032387
:101BA0001B049A43074B1A6306E0064A126B032391
:101BB0009B049A43034B1A63024A126B0243014B84
:101BC0001A637047001002400549096B8022914357
:101BD000034A11631146096B01431163704700000A
:101BE0000010024038B5002000900024002500BFFE
:101BF0001120FFF71FFF05460098401C00900521AB
:101C000009030098884201D0002DF1D01120FFF780
:101C100011FF002801D0012400E00024204638BD37
:101C200070B502460B46FF20002115E0555C684068
:101C300008240DE080250540002D05D04500FF2635
:101C400032367540E8B201E04506280E651EECB25A
:101C5000002CEFDC4D1CE9B29942E7DB70BD0000BF
:101C600070B504462046FEF7E5FB06460349FEF73D
:101C7000EDFA05460249FEF726FB70BD0000C8429A
:101C800000FF7F47F8B504462046FEF7D3FB074622
:101C90000549FEF7DBFA06460449FEF714FB054644
:101CA0000349FEF7CBFAF8BD00002F4300FF7F4742
:101CB00000003442F8B505460E4614463146284623
:101CC000FFF7AEFF0746A74201D00220F8BD002073
:101CD000FCE7FFB581B006460F461D46002D02D039
:101CE000012D10D107E0394630460A9B039A00F0D7
:101CF00011F8044609E0394630460A9B039A00F081
:101D000055F8044601E0802400BF00BF204605B01E
:101D1000F0BD0000FFB583B005460E46174600F043
:101D20002BF90446002C19D1002F0ED0012F06D01C
:101D3000022F10D11C4800F02FF904460DE01A487C
:101D4000C01E00F029F9044607E017480A3800F0E1
:101D500023F9044601E0802400BF00BF002C02D11B
:101D600000F0FEF80446002C05D1002102A8069AD6
:101D700000F0BAF80446002C05D10022012101A888
:101D800000F0B2F8044600F003F9002C09D16846CF
:101D90000089FFF777FF286068468088FFF760FFBB
:101DA0003060204607B0F0BD102C0000FFB583B0B6
:101DB00006460F461D4600F0DFF80446002C1AD1F7
:101DC000059800280ED0012806D0022810D12448FA
:101DD00000F0E2F804460DE021480B3800F0DCF892
:101DE000044607E00920800200F0D6F8044601E02E
:101DF000802400BF00BF002C13D109E000F0B0F830
:101E00000446002C00D108E07D20C000FEF7A0FFB2
:101E10002846691ECDB20028F0D100BF002D00D1A8
:101E20000424002C0BD10022114602A800F05CF81B
:101E300004430022012101A800F056F8044300F0F9
:101E4000A7F8002C09D168460089FFF71BFF306016
:101E500068468088FFF704FF3860204607B0F0BD71
:101E6000162400001CB504460120800200900021C9
:101E700068460171C17169461A48FFF719F90120D6
:101E80000003009001216846017100218171032146
:101E900041710021C17169461248FFF709F901201B
:101EA00040071049886103204002009001216846E4
:101EB00001718171032141710021C17169460920BD
:101EC000C006FFF7F5F8012080020921C9068861E4
:101ED00040108861204600F033F80120400301499A
:101EE00088611CBD00040048FEB505460E46174635
:101EF0003A46002101A8FFF71DFA0446002C06D13E
:101F00000022114601A80130FFF714FA0446002C04
:101F100005D1002231466846FFF70CFA0446002C32
:101F200006D168460278022101A8FFF7C3FE0446E5
:101F30006946087900024979084328802046FEBD99
:101F40004106090E044A1170114609780122114315
:101F5000024A1170704700002B0000202C00002066
:101F600010B5FFF73EFA03480078FFF796FA0446EB
:101F7000204610BD2C00002010B5FFF732FA0348B0
:101F80000078FFF78AFA0446204610BD2B00002097
:101F900010B5FFF748FA10BD70B504462012FFF7E0
:101FA0007CFA0546E0B2FFF778FA0543284670BD93
:101FB0007047704710B5C820FEF7C0FE07221749CA
:101FC000174800F039FEC820FEF7B8FE092215496F
:101FD000154800F031FEC820FEF7B0FE0922134973
:101FE000134800F029FEC820FEF7A8FE09220F4979
:101FF000104800F021FEC820FEF7A0FE09220E497D
:102000000E4800F019FE6420FEF7B8FE4420FFF7EA
:1020100029FF3220FEF7B2FE10BD0000DB360008BB
:10202000004C00403F3700080048004024370008BB
:102030000050004000380140003700080014014003
:102040000CB500200190009031480068012109047E
:1020500008432F49086000BF2D480068012149044A
:10206000084000900198401C01900098002804D17D
:102070000521090301988842EED125480068012115
:1020800049040840002802D00120009001E000200F
:1020900000900098012839D111201E4908601C4881
:1020A00040681B49486008464068486008464068E8
:1020B0007F21C903884316494860084640680521C6
:1020C00009040843124948600846006801210906CE
:1020D00008430F49086000BF0D4800680121490608
:1020E00008400028F8D00A48406880088000084965
:1020F000486008464068022108430549486000BF1F
:10210000034840680C2108400828F9D10CBD0000A4
:10211000001002400020024010B57D21C900104887
:102120000068FEF701F80446601E0E49884201D996
:1021300001200CE0601E0C4948610321081FFFF7D5
:10214000A9FA0020084988610720086100200028BA
:1021500001D000BFFEE70021481EFFF79BFA10BD2B
:1021600000000020FFFFFF0000E000E004480068DE
:10217000002804D002480068401E014908607047EA
:102180003C00002010B51B48006801210843194994
:1021900008600846406818490840164948600846E3
:1021A0000068164908401349086008460068012184
:1021B000890488430F490860084640683F210904A4
:1021C00088430C4948600846C06A00090001C8629B
:1021D0000846006BFF2154318843064908630846CE
:1021E000406B40084000486300208860FFF728FFEC
:1021F00010BD0000001002400CB8FF08FFFFF6FE03
:1022000010B50121134800F03FF8002820D001212B
:10221000104800F028F810480078002809D001285C
:102220000ED0022813D101200B4908700B49087009
:102230000DE002200849087001200849087006E0F6
:1022400000200549087001200449087000BF00BF44
:1022500010BD0000001000402500002026000020D6
:10226000CA4302827047CA4302827047002904D0E1
:10227000028801231A43028003E00288014B1A40BE
:1022800002807047FEFF000030B5024600200023A8
:102290000024158A0D402B4695890D402C46002BB5
:1022A00003D0002C01D0012000E0002030BD002A26
:1022B00003D083890B43838102E083898B4383812D
:1022C000704700000EB501211020FFF731FA0B48CE
:1022D00001900B48694608800A4800F015F8012172
:1022E0000848FFF7BDFF012211460648FFF7DFFF50
:1022F00001210448FFF7BAFF0EBD0000BF5D0000DA
:102300001F4E00000010004000220288154B98422A
:1023100006D001239B07984202D0134B984203D169
:10232000124B1A404B881A43114B984203D0114B61
:102330001A400B891A4302804B68C3620B880385DD
:10234000084B984208D00C4B984205D00B4B984252
:1023500002D00B4B984201D18B7A038601238382F2
:1023600070470000002C0140000400408FFF000077
:1023700000100040FFFC000000400140004401400C
:102380000048014010B500F003F8FFF79BFF10BDB7
:1023900008B511216846017000214170012181704A
:1023A000FFF740F908BD000010B50B490B4800F0DD
:1023B000C5FA00280FD00849084800F0C7F90021E5
:1023C0000748FEF73BFC402005490839C860012159
:1023D0000348FEF733FC10BD04010400003801403F
:1023E0000800024010B50749074800F0A7FA002886
:1023F00007D0054800F078FBC4B20249024800F05B
:10240000A5F910BD050105000044004010B5B04914
:10241000B04800F093FA00280FD0AD49AD4800F065
:1024200095F90021AC48FEF709FC4020AA49303953
:1024300048630121A848FEF701FCA549A74800F020
:102440007DFA00280FD0A249A44800F07FF90021AE
:10245000A348FEF7F3FB8020A1491C390862012143
:102460009F48FEF7EBFB9A499E4800F067FA002868
:1024700011D097499B4800F069F90021964828300F
:10248000FEF7DCFB402094491031C86101219248DD
:102490002830FEF7D3FB9449944800F04FFA002807
:1024A00013D0924800F020FBC1B29148914A1278B3
:1024B000815490480078401C8E4908700846007886
:1024C00008708949894800F041F98A480078401E1F
:1024D0008749085CFF2805D186480078401E864958
:1024E000087053E083480078401E83490978491CEE
:1024F00088420CD17F480078401E7D49085C8628C0
:1025000005D17C480078401E7C4908703EE079483F
:102510000078401E79490978C91D884236D10024C7
:102520007649087804E07249095C0919CCB2401C6C
:1025300072490978C91D8842F5DBE043401CC4B2EA
:102540006B496E480078C01D085C844218D108466B
:102550006A490978405C862812D165496748007845
:10256000401C085C0102624A64480078801C105CD0
:102570000818634948610846416962A000F072FB8F
:102580000020634908705B49087000BF56496148E4
:1025900000F0D4F9002815D053495E4800F0CEF978
:1025A00000280ED05B4800F09FFAC4B200BF802123
:1025B000594800F0B9F90028F9D04B49554800F0C6
:1025C000C5F800BF4249554800F0B8F900287ED050
:1025D0003F49524800F0BAF8002141481430FEF754
:1025E0002DFB80203E491C39486301213C481430B2
:1025F000FEF724FB0A224A494AA0FDF7BFFD002846
:102600001CD14748807A3038002806D0012808D0ED
:1026100002280AD0032810D10BE00020444908709A
:102620000BE001204249087007E002204049087091
:1026300003E003203E49087000BF00BF0A2238496A
:102640003CA0FDF79BFD00281CD13548807A30382E
:10265000002806D0012808D002280AD0032810D16B
:102660000BE00020324908700BE00120304908706F
:1026700007E002202E49087003E003202C4908706F
:1026800000BF00BF082226492DA0FDF777FD0028D6
:102690001DD12348007A3038002806D0012809D0FF
:1026A00002280BD0032811D10CE00020204908702B
:1026B0000CE00CE001201E49087007E002201C49D4
:1026C000087003E003201A49087000BF00BF10BD66
:1026D000040104000048004030000240004C00406B
:1026E0001C04024000500040050105000014014098
:1026F000D40100202700002028000020290000200D
:102700005C000020636F323A2025640D0A0000004F
:102710002A0000200018014000440040001C014035
:10272000940200200D0A2B5354415455533A000093
:10273000240000200D0A5E5354415455533A0000C2
:102740005E5354415455533A0000000010B5002325
:1027500000220B0C01249C402246026210BD00297D
:1027600004D0026801231A43026003E002685208A1
:10277000520002607047000000B587B04B20C001D6
:102780000190002002900390049006900C20059088
:1027900001A9574800F01AF900225649544800F0A0
:1027A000F4F801215248FFF7DAFF4B20C0010190F5
:1027B000002002900390049006900C20059001A93F
:1027C0004D4800F003F900224A494B4800F0DDF87B
:1027D00001214948FFF7C3FF4B20C00101900020B1
:1027E00002900390049006900C20059001A94348A4
:1027F00000F0ECF800223F49404800F0C6F8012103
:102800003E48FFF7ACFF4B20C00101900020029032
:102810000390049006900C20059001A9384800F020
:10282000D5F800223349364800F0AFF8012134488A
:10283000FFF795FF4B20C00101900020029003900C
:10284000049006900C20059001A92E4800F0BEF8D7
:10285000002228492B4800F098F801212948FFF769
:102860007EFF4B20C0010190002002900390049055
:1028700006900C20059001A9234800F0A7F801223A
:102880001C49214800F081F801211F48FFF767FF2C
:10289000E1204002019000200290039004900690F5
:1028A0000C20059001A9194800F090F80122114967
:1028B000164800F06AF800211448FFF750FF4B203B
:1028C000C0010190002002900390049006900C201B
:1028D000059001A90E4800F079F8002205490C483E
:1028E00000F053F801210A48FFF739FF07B000BD97
:1028F0000044004005010500003801400048004048
:10290000004C0040005000400014014000180140FD
:10291000001C0140002A03D083680B43836002E05F
:1029200083688B438360704702460020D3690B4065
:10293000002B01D0012000E00020704770B5024656
:102940000B4600240021002500201E04350ED9B2BC
:1029500001268E403146012D02D11668314006E035
:10296000022D02D15668314001E0966831401C0CBE
:102970000126A6403446D6693440002903D0002CF5
:1029800001D0012000E0002070BDF8B5034600240E
:10299000002600960025002018460E04340ECEB204
:1029A00000960127009EB7403D46022C01D1001D34
:1029B00002E0032C00D10830002A03D006682E4321
:1029C000066002E00668AE430660F8BDF0B58BB065
:1029D00004460D46002700200A9000262068400883
:1029E000400020606668032109033046884306469C
:1029F000A8680643666026682D480640E96868684E
:102A000008432969084306432660A6680321090292
:102A100030468843064668690643A6606846FEF766
:102A2000E3FE2448844202D106980A900DE0224831
:102A3000844202D107980A9007E02048844202D1DC
:102A400008980A9001E002980A9020680121C903C1
:102A5000084000280CD029680A9A5000FDF764FB52
:102A6000074629680A9A5000FDF75EFB0E4609E00A
:102A700029680A98FDF758FB074629680A98FDF768
:102A800053FB0E4628684008B04200D87F1C2068DF
:102A90000121C9030840002806D03807460F3846F0
:102AA0000749084030430746A7810BB0F0BD00003E
:102AB000F3E9FFFF003801400044004000480040B7
:102AC000F0FF000010B501212F204004FEF720FE8A
:102AD00001210F204004FEF72BFE01210148FEF7E3
:102AE00037FE10BDE14000000146888CC005C00DD6
:102AF0007047CA05D20D0285704700000EB5082048
:102B000020494022204B0092019102901F4A01214E
:102B10001C48083000F056F81D481A4940221D4B49
:102B20000092019102901C4A01211648303000F0B9
:102B300049F81A481A4980221A4B009201910290D2
:102B4000194A022116481C3000F03CF817480D497C
:102B50004022174B009201910290164A0121094828
:102B6000583000F02FF814480D498022134B009282
:102B700001910290124A02210948303000F022F8F7
:102B80000EBD00000000024094000020003801400B
:102B9000000A0020D400002000480040B0000010CF
:102BA0000004024014010020004C004000000C40D2
:102BB0009401002000500040000F002094020020EB
:102BC000001C0140F0B58BB007460D4614461E466A
:102BD00001212846FEF79CFD2046243000900196F6
:102BE000002002901098039000200490802005900F
:102BF0000020069007900890012000030990002013
:102C00000A9069463846FEF741F801213846FEF73A
:102C100015F812991198FEF759F801220549204636
:102C2000FFF7B3FE012240212046FFF773FE0BB0F1
:102C3000F0BD00000401040070B506460C461546C0
:102C40000BE02178641C3046FFF753FF00BF802162
:102C50003046FFF769FE0028F9D028466D1E00288F
:102C6000EFD170BD0FB410B503A9044B044A02980C
:102C700000F0E8F810BC08BC04B018477D35000827
:102C8000580000202021020C01D010211046020A19
:102C900001D010460839020901D01046091F8208E8
:102CA00001D01046891E420801D0881E7047081ABC
:102CB000704702E008C8121F08C1002AFAD1704705
:102CC0007047002001E001C1121F002AFBD17047AC
:102CD000F0B51FB486B00998089A030D002102438D
:102CE00014D05148514A181850430514119801281E
:102CF00010981AD0281A401C00264D4F4D490096B6
:102D000001910490002812DA444211E01198012444
:102D100049A3012801D11098C1430698119A8460F3
:102D20000360C26041600BB0F0BD4042E4E704467E
:102D3000210500203F4A001C51410391029012E0FE
:102D4000E00707D032463B4601990098FDF764FD45
:102D50000191009032463B4610461946FDF75CFD56
:102D600006460F466410002CEAD10498039B002805
:102D7000029A0999089806DAFDF74EFD019B009A20
:102D8000FDF74AFD05E0FDF7DDFA019B009AFDF72E
:102D9000D9FA04460E460022284BFDF7C5FD03D89C
:102DA0000020C043014607E00022254B2046314663
:102DB000FDF780FCFDF798FD102409E0002C0ADBEC
:102DC0000A220023FDF7A6FB079B30321A55641E2A
:102DD00002460A43F2D11122641C079B121B1C19E4
:102DE000119B012B03D0012308430ED10AE00843B5
:102DF00004D0112010900020119077E71098151A38
:102E00006D1E0BE01098824202DD00236D1C03E072
:102E1000824201DA00236D1E002BEED00698119934
:102E20008260C16030C07EE701FCFFFF104D0000F2
:102E3000000014400000F03F300000000000F043AC
:102E40000000E03FFFB597B00646002518E22528B0
:102E500077D100242746FD49049400E00443761C02
:102E600032780120203A90400842F7D130782A2861
:102E70000ED00222307801463039092916D804993B
:102E80000A235943303940181443761C0490F1E763
:102E9000189802C804911890002904DA0120400310
:102EA00004434842049002200443761C30782E28C4
:102EB00014D1042004437078761C2A2809D118986C
:102EC000761C80C8189009E00A214F43303FC7198B
:102ED000761C3078014630390929F5D930786C28CC
:102EE00010D006DC4C281AD068280ED06A2817D1DA
:102EF00004E0742813D07A2812D110E00120400594
:102F000004430CE00121090501E0032109050C43FC
:102F10007178814203D1012000052418761C761CAB
:102F20003078119066280BD013DC58287DD009DC4E
:102F300000287BD04528F6D04628F4D047281AD15F
:102F4000A5E118E0632835D0642870D0652812D137
:102F50009DE170286CD008DC6728F1D069287BD00F
:102F60006E280DD06F2806D1BAE073282ED07528B0
:102F700071D0782859D01A9A199990476D1C7EE122
:102F80006002400F022809D003280DD004281898A9
:102F900001680DD00D60001D189070E11898EA17B7
:102FA00001680D604A60F6E7189801680D80F2E745
:102FB0000D70F0E718986A4601781172001D18909C
:102FC0000020507202A80090012005E0189802C865
:102FD000189000200091C04361070DD5002101E049
:102FE0000199491C0191B94212DA8142F8DB009A39
:102FF000515C0029F4D10BE0002101E00199491C4A
:1030000001918142FADB019A0099895C0029F5D18E
:10301000019904981A9B471A21463846199A00F0DC
:1030200097FA0199401945180BE04FE02CE113E0A5
:103030004EE0009800990078491C00911A9A19995D
:1030400090470198401E0190401CF2D1214638461D
:103050001A9B199A10E137E00A2000210090019193
:103060006002410F022907D0189A01CA1892C217AC
:103070009446032908D00AE01898C01DC108C90069
:1030800005C91891944607E000B2C2179446042976
:1030900002D140B2C1178C4600226146944506DA3F
:1030A0000A460021404291418C462D2102E0210533
:1030B00004D52B216A461173012103E0E10701D0F9
:1030C0002021F7E7029155E00A200AE0102008E0ED
:1030D000102000900021042004430191082703E000
:1030E00008200021019100906002410F022907D0C1
:1030F000189A01CA189200229446032908D008E0C1
:103100001898C01DC108C90005C91891944603E06C
:1031100080B2042900D1C0B200210291210729D533
:103120001199702906D0009A1021019B4A401A4338
:1031300005D00EE040216A461173012108E0614686
:10314000014306D030216A4611731199517302214F
:103150000291009A0821019B4A401A430AD1614614
:10316000014301D1610705D530216A461173012160
:103170007F1E02911199582904D035A10E910DA9F5
:103180000D910DE037A1F9E76146019B009AFDF72B
:10319000C1F90E9B8C469B5C0D9A521E0D921370CA
:1031A00061460143F0D10D9805A9081A203001901D
:1031B000600703D501200004844300E00127019843
:1031C000874201DD381A00E0002001990090411883
:1031D000029809180498401A0490E00306D4214686
:1031E0001A9B199A049800F0B3F94519002706E0D4
:1031F00003A81A9AC05D199990476D1C7F1C02980C
:103200008742F5DBE0030CD521461A9B199A0498F6
:1032100000F09EF9451904E01A9A30201999904758
:103220006D1C0099481E00900029F5DC08E00D98FF
:103230000D990078491C0D911A9A199990476D1CA7
:103240000199481E01900029F1DC63E10928010081
:10325000303132333435363738396162636465660C
:1032600000000000303132333435363738394142CE
:10327000434445460000000000F05AF94519761C09
:103280003078002800D0E2E528461BB0F0BD60078A
:1032900000D406271898C01DC108C90048680A68EC
:1032A0000831C30FDB071891190001D09CA108E079
:1032B000210501D59BA104E0E10701D09AA100E01E
:1032C0009AA1430011985B08109165280CD006DC88
:1032D000452809D046281DD0472841D141E066281D
:1032E00018D067283CD13CE00021112F01DB1120D0
:1032F00000E0781C0191009008A911A8FFF7E8FCF4
:10330000139905910021119A15927F1C129801972B
:10331000009150E00120C00703900120019008A90E
:10332000009711A8FFF7D4FC139A14990592002274
:10333000119B009212981593059A0192002901D0D1
:10334000104602E0791C40180190381A01D5019806
:1033500004E04042401E0090781C0190C01B029087
:1033600043E0012F00DA01270021112F01DD112098
:1033700000E038460191009008A911A8FFF7A8FCC9
:1033800013990591119A00211298159200910197B5
:1033900021070CD40599B94201DB019900E00191A4
:1033A000012904DD159A491E515C302906D0B84226
:1033B00001DA011D05DA0121029115E00199491E8A
:1033C000EDE7002805DC0099411800910199091AE0
:1033D00003E0019A411C914200DD01910099401ADD
:1033E000401C02900120C0070390200706D40299D8
:1033F0000198814202DB0020C04302900020694610
:10340000C87707AF012103980337C907884224D042
:10341000022011902B201290039800280CDA4042D1
:1034200003902D20129007E00A210398FCF77CFE00
:1034300030317F1E039039701199481E1190002978
:10344000F2DC03980028EFD1791E129808703078CA
:10345000202108404530BF1E387006A8C01BC01D83
:10346000039010980078002800D00120019941189D
:103470000298C0170918039809180498401A401EAA
:103480000490E00306D421461A9B199A049800F090
:103490005FF8451910980078002803D01A9A1999F6
:1034A00090476D1CE00324D521461A9B199A049875
:1034B00000F04EF845191CE00098002807DB009941
:1034C0000598884203DD1598405C199901E0199927
:1034D00030201A9A904700986D1C401C009002986A
:1034E000401E0290002804D11A9A2E201999904764
:1034F0006D1C0199481E01900029DDDC05E038783B
:103500001A9A7F1C199990476D1C0399481E0390C5
:103510000029F4DC21461A9B199A0498ACE60000B5
:103520002D0000002B000000200000000000000023
:10353000F8B5044600251E461746880404D405E065
:1035400039462020B0476D1C641EF9D52846F8BDC9
:10355000FFB50446002581B01E46C80301D53027BB
:1035600000E02027880404D505E038460399B047D9
:103570006D1C641EF9D5284605B0F0BD70B5044633
:103580000D46E1B20548FFF7B4FA00BF80210348B9
:10359000FFF7CAF90028F9D0204670BD004400406A
:1035A000FEF7E6F80120FEF781FAFEF71BFB044662
:1035B000012C34D1FDF732FC0120FDF741FC002045
:1035C000FEF7C2FAA1048810FEF7ACFA0120FEF75C
:1035D00095FA00BF1920FEF72DFA0028FAD0022034
:1035E000FEF7C0FA00BFFEF749FA0828FBD1002019
:1035F000FEF74CFA0020FEF76FFA01200007FEF7F5
:10360000BFFA01204007FEF7BBFA03200007FEF7D0
:10361000B7FA1020FEF752FA8020FEF7D5FAFEF72F
:103620007BFDFFF74FFAFDF719FCFFF7A5F8FDF753
:10363000B6FF6420FDF7A2FBFF2101310920C0067F
:10364000FDF7AAFD6420FDF799FBFF210131092058
:10365000C006FDF7A3FDFFF751FAFEF793FE1548EC
:10366000FDF76CFBFEF7A6FC13490620FDF75CFF97
:1036700012A0FFF7F7FA1BE014480078012815D1D3
:1036800013480078002804D0012805D0022809D169
:1036900005E0FEF73BF805E0FDF7B4FA02E0FDF7C0
:1036A0002FFB00BF00BF002008490870FDF758FF3E
:1036B000E2E70000B80B0000FF0F00004445425550
:1036C0004720546573740D0A000000002600002096
:1036D00025000020424DE200000171424DE1000052
:1036E0000170424DE100010171424DE4000001739F
:1036F000424DE400010174FF0186000000000079E2
:10370000FF019900000007D08FFF0199000000130E
:1037100088CBFF019900000027102FFF01860000D1
:1037200000000079FF0178040000000083FF01869B
:10373000030000000084FF0186000000000079FF04
:103740000178410000000046FF01784000000000C1
:103750004700000074370008000000205C000000F3
:10376000B22C0008D03700085C000020BC06000026
:10377000C22C0008006CDC02000000000000000009
:103780000102030406070809000000000102030407
:1037900001020304060708090301010000000000FC
:1037A0000000000000000000000000000000000019
:1037B0000000000000000000000000000000000009
:1037C00000000000000000000000000000000000F9
:04000005080000BD32
:00000001FF
